S01A000064656D6F70726F675F73746D3332663230372E7372656396
S3150800800000090020619E00089D9E0008A19E0008A8
S31508008010A59E0008A99E0008AD9E00080000000065
S31508008020000000000000000000000000B19E0008EB
S31508008030B59E000800000000B99E00087B9800085D
S31508008040BD9E0008C19E0008C59E0008C99E00087E
S31508008050CD9E0008D19E0008D59E0008D99E00082E
S31508008060DD9E0008E19E0008E59E0008E99E0008DE
S31508008070ED9E0008F19E0008F59E0008F99E00088E
S31508008080FD9E0008019F0008059F0008099F00083B
S315080080900D9F0008119F0008159F0008199F0008EA
S315080080A01D9F0008219F0008259F0008299F00089A
S315080080B02D9F0008319F0008359F0008399F00084A
S315080080C03D9F0008419F0008459F0008499F0008FA
S315080080D04D9F0008519F0008559F0008599F0008AA
S315080080E05D9F0008619F0008659F0008699F00085A
S315080080F06D9F0008719F0008759F0008799F00080A
S315080081007D9F0008819F0008859F0008899F0008B9
S315080081108D9F0008919F0008959F0008999F000869
S315080081209D9F0008A19F0008A59F0008A99F000819
S31508008130AD9F0008B19F0008B59F0008B99F0008C9
S31508008140BD9F0008C19F0008C59F0008C99F000879
S31508008150CD9F0008D19F0008D59F0008D99F000829
S31508008160DD9F0008E19F0008E59F0008E99F0008D9
S31508008170ED9F0008F19F0008F59F0008F99F000889
S31508008180FD9F0008EE11AA5570B5040000250020D1
S31508008190002C01D10120C9E094F83C00002805D143
S315080081A0002084F83D00200000F0AEFA022084F892
S315080081B03C002068006830F00200216808602068EA
S315080081C0006850F001002168086000F0BBFA06005C
S315080081D020684068C0070CD400F0B4FA801B0B284E
S315080081E0F6D3032084F83C00002084F83D000320E1
S315080081F09CE020684068C00740F18B80A069012890
S3150800820006D12068006850F080002168086005E003
S315080082102068006830F0800021680860E06901285D
S3150800822006D12068006850F040002168086005E023
S315080082302068006830F0400021680860206A01283C
S3150800824006D12068006850F020002168086005E023
S315080082502068006830F0200021680860606A0128FC
S3150800826006D12068006850F010002168086005E013
S315080082702068006830F0100021680860A06A0128AC
S3150800828006D12068006850F008002168086005E0FB
S315080082902068006830F0080021680860E06A012854
S315080082A006D12068006850F004002168086005E0DF
S315080082B02068006830F0040021680860A168E0685A
S315080082C0014320690143606901436068401E014318
S315080082D02068C1612068006840084000216808607D
S315080082E000F030FA060020684068C0070CD500F098
S315080082F029FA801B0B28F6D3032084F83C000020BB
S3150800830084F83D00032011E020684068C00700D4C7
S315080083100125012D06D100202064012084F83C00A7
S31508008320002003E0042084F83C00012070BD70B4EE
S31508008330002001204A6910FA02F2DFF8E8301868CE
S3150800834050F001001860186830F47C5018601868FE
S315080083504C6A50EA04201860DFF8CC402068904345
S315080083602060C869002817D1DFF8C0000568954362
S315080083700560DFF88803CD684E68B6B256EA05464A
S315080083804D6940F835604D6900EBC5008D680E688B
S31508008390B6B256EA05464660C869012816D123488A
S315080083A0056815430560DFF854030D684E68B6B2D4
S315080083B056EA05464D6940F835604D6900EBC5003B
S315080083C08D68CE68B6B256EA0546466088690028C2
S315080083D005D1DFF82C0305689543056004E0DFF84E
S315080083E020030568154305600869002804D1DFF8ED
S315080083F014030568954305600869012804D1DFF868
S315080084000403056815430560086A012802D1206837
S31508008410024322601868400840001860002070BCBB
S3150800842070470000006600401C6600400C6600406D
S31508008430F8B505000E001400002000203000C0B278
S31508008440002811D195F83C0022280BD095F83C005D
S31508008450422807D095F83C00622803D095F83C00DE
S31508008460722801D1022048E13000C0B2012811D19A
S3150800847095F83C0032280BD095F83C00522807D0D6
S3150800848095F83C00622803D095F83C00722801D183
S31508008490022032E195F83D00012801D102202CE1A5
S315080084A0012085F83D003000C0B2002818D195F8A3
S315080084B03C00122804D0322806D0522808D00BE0F7
S315080084C0422085F83C0023E0622085F83C001FE046
S315080084D0722085F83C001BE0222085F83C0017E056
S315080084E095F83C00122804D0222806D0422808D045
S315080084F00BE0522085F83C000AE0622085F83C0033
S3150800850006E0722085F83C0002E0322085F83C003F
S3150800851000F018F907003000C0B2002804D1286816
S31508008520C06810F0030003E02868006910F0030033
S31508008530002811D114F1010FEDD0002C04D000F061
S3150800854001F9C01B8442E6D2032085F83C000020CE
S3150800855085F83D000320D0E03000C0B2002801D1E4
S31508008560696B00E0A96B28683200D2B21201104488
S31508008570D0F8B00110F0040088608868002809D196
S3150800858028683200D2B212011044D0F8B001400D6A
S31508008590086008E028683200D2B212011044D0F808
S315080085A0B001C008486028683200D2B212011044EF
S315080085B0D0F8B00110F00200C86028683200D2B2C4
S315080085C012011044D0F8B40110F00F0008612868B1
S315080085D03200D2B212011044D0F8B401C0F3072019
S315080085E0C8613000C0B2086228683200D2B21201EF
S315080085F01044D0F8B801087528683200D2B21201C2
S315080086001044D0F8B801000A487528683200D2B27A
S3150800861012011044D0F8B801000C88752868320099
S31508008620D2B212011044D0F8B801000EC8752868F5
S315080086303200D2B212011044D0F8BC01087628687C
S315080086403200D2B212011044D0F8BC01000A4876B2
S3150800865028683200D2B212011044D0F8BC01000CCE
S31508008660887628683200D2B212011044D0F8BC01CC
S31508008670000EC8763000C0B2002803D12020296831
S31508008680C86002E0202029680861F6B2002E18D1D9
S3150800869095F83C00422804D0622806D0722808D0F3
S315080086A00BE0122085F83C0023E0322085F83C00D8
S315080086B01FE0522085F83C001BE0012085F83C00AD
S315080086C017E095F83C00522804D0622806D0722894
S315080086D008D00BE0122085F83C000AE0222085F835
S315080086E03C0006E0422085F83C0002E0012085F8BF
S315080086F03C00002085F83D000020F2BD40660040A1
S315080087000466004014660040704730B4002513E044
S3150800871050F8042BD30744BFA9F101039A18091F7F
S31508008720042942F8045BFAD213468C0744BF158025
S315080087309B1CC90748BF1D7050F8041B0029E7D1C8
S3150800874030BC704701480068704700BFF800002039
S31508008750F8B50400002C01D1012079E12078C00782
S315080087603FD5DFF8F404016811F00C01042909D09B
S31508008770006810F00C0008280ED1DFF8E004006845
S31508008780400209D5DFF8CC040068800329D5606863
S31508008790002826D101205BE16068DFF8D014087054
S315080087A0606800280ED0FFF7CDFF0500DFF8A404A7
S315080087B00068800315D4FFF7C5FF401B6528F5D36D
S315080087C0032045E1FFF7BEFF0500DFF888040068CF
S315080087D0800306D5FFF7B6FF401B6528F5D30320AF
S315080087E036E12078800725D5DFF86C04016811F09A
S315080087F00C0F09D0006810F00C00082833D1DFF8F8
S315080088005C04006840022ED4DFF848040168890732
S3150800881004D5E168012901D0012019E101685FF05A
S31508008820F852B2FA82F231F0F801236913FA02F229
S3150800883011430160207800075ED56069002848D09A
S315080088400120DFF82C140860FFF77CFF0500DFF82D
S315080088501004006880074FD4FFF774FF401B0328F5
S31508008860F5D30320F4E0E06800281FD00120DFF8E4
S3150800887004140860FFF766FF0500DFF8D8030168EF
S31508008880890706D4FFF75EFF401B0328F5D30320AC
S31508008890DEE001685FF0F852B2FA82F231F0F801D0
S315080088A0236913FA02F211430160C3E70020DFF8D7
S315080088B0C4130860FFF746FF0500DFF89803006851
S315080088C08007B7D5FFF73EFF401B0328F5D30320E3
S315080088D0BEE00020DFF898130860FFF733FF0500B5
S315080088E0DFF87C030068800706D5FFF72BFF401BDF
S315080088F00328F5D30320ABE02078400744D50020B1
S315080089000090DFF87403016851F080510160006837
S3150800891010F0805000900098DFF86063306850F4DB
S3150800892080703060FFF70EFF05003068C00506D47A
S31508008930FFF708FF401B0328F7D3032088E0DFF87A
S315080089404053A0682870A06800280ED0FFF7FAFEEA
S3150800895006002868800717D4FFF7F4FE801B41F24B
S3150800896089318842F5D3032072E0FFF7EBFE060053
S315080089702868800708D5FFF7E5FE801B41F2893194
S315080089808842F5D3032063E0A06900285FD0DFF8AA
S31508008990C802006810F00C00082856D0A069022802
S315080089A040D1DFF8E06200203060FFF7CBFE070019
S315080089B0DFF8A0522868800106D5FFF7C3FEC01B62
S315080089C06528F5D3032043E0DFF8BC02B0FA80F14E
S315080089D04FF44040B0FA80F2F020B0FA80F3E7692D
S315080089E0206A0743606A10FA01F13943A06A400811
S315080089F0401E10FA02F21143E06A10FA03F3194313
S31508008A00DFF85802016001203060FFF79BFE040082
S31508008A10286880011BD4FFF795FE001B6528F7D34D
S31508008A20032015E00020DFF85C120860FFF78AFED5
S31508008A300400DFF820020068800108D5FFF782FEEF
S31508008A40001B6528F5D3032002E0012000E0002082
S31508008A50F2BD2DE9F04104000E00002C01D10120E1
S31508008A609AE0DFF82852286810F00F00B04207D2C3
S31508008A702E70286810F00F00B04201D001208BE05C
S31508008A802078800719D52078400705D5DFF8C80172
S31508008A90016851F4E05101602078000705D5DFF838
S31508008AA0B801016851F460410160DFF8AC110A6849
S31508008AB032F0F002A06802430A602078C00735D574
S31508008AC06068012806D1DFF88C010068800312D49B
S31508008AD0012061E06068022806D1DFF878010068A5
S31508008AE0800108D4012057E0DFF868010068800794
S31508008AF001D4012050E0584F396889088900606818
S31508008B0001433960FFF71EFE8046386810F00C00F6
S31508008B106168B0EB810F09D0FFF714FEB0EB0800CF
S31508008B2041F289318842F0D3032035E0286810F0F5
S31508008B300F00864207D22E70286810F00F00B04248
S31508008B4001D0012028E02078400706D542490A6866
S31508008B5032F4E052E06802430A602078000707D53D
S31508008B603D48016831F46041226951EAC201016059
S31508008B7000F014F8384909685FF07062B2FA82F2B8
S31508008B80434B11F0F001D140595CC84036490860A2
S31508008B90002000F083F80020BDE8F08110B5002021
S31508008BA00020002000202C48006810F00C00002847
S31508008BB004D0042804D0082804D025E0294824E055
S31508008BC0344822E0254C226812F03F022068400211
S31508008BD009D52068C0F388102E49A1FB000100239F
S31508008BE000F070F808E02068C0F388101D49A1FB62
S31508008BF00001002300F066F82168C1F30141491C11
S31508008C004900B0FBF1F000E0164810BD16480068B0
S31508008C10704780B5FFF7FAFF0F4909685FF46012DD
S31508008C20B2FA82F21C4B11F4E051D140595CC840AB
S31508008C3002BD80B5FFF7EAFF074909685FF4E0223D
S31508008C40B2FA82F2144B11F46041D140595CC84023
S31508008C5002BD0000003802400838024004380240CD
S31508008C60743802400024F400000000200238024054
S31508008C70800E4742000047424038024000700040DC
S31508008C8070380240600047420000FE03003C024084
S31508008C90789E000840787D01949E000810B504006F
S31508008CA0074800684FF47A71B0FBF1F000F090F9CC
S31508008CB0002221005FF0FF3000F079F9002010BD96
S31508008CC000000020BBBBE1B1B2F5803F80F07E809A
S31508008CD0022A1ED98C46B1FBF2F102FB11C31B0412
S31508008CE043EA1043B3FBF2FC02FB1C3380B240EAB2
S31508008CF00343B3FBF2F002FB103240EA0C400023B8
S31508008D007047022A05D98446B0FBF2F002FB10C26E
S31508008D1070474AB105D100F0010249085FEA300000
S31508008D20704700220023704700F090B90B0002003C
S31508008D30002100207047904271EB030CF6D3B3F57F
S31508008D40803F2FD2F0B5B3FA83F7B1FA81F4A7F1D1
S31508008D500F0E3D1B5340CEF1200602FA0EF2F341E8
S31508008D605340B5F10F0746D80F3C2C444140C4F197
S31508008D702006A040F1414140B1FBF3F603FB161172
S31508008D80A2FB0645001BA94102D2761E801859414E
S31508008D9080EA010221FA0EF362FA0EF200215A4025
S31508008DA03046F0BD30B4B1FBF3FC03FB1C11A2FB4B
S31508008DB00C45001BA94103D2ACF1010C801859419E
S31508008DC030BC02460B46604600217047B2F1807FF0
S31508008DD065D3F0B5B2FA82F7B1FA81F4C7F10F0696
S31508008DE03D1B22FA06F307F1110EF24120355A40CF
S31508008DF0B5F10F07B8D94140C4F12006A040F141AA
S31508008E004140B1FBF3FC03FB1C11A2FB0C45001B04
S31508008E10A94103D2BCF1010C801859410F2F12D376
S31508008E200F3FC90341EA5041B1FBF3F603FB1611A4
S31508008E30A2FB0645D4EBC030A94102D2761E8018A3
S31508008E40594146EACC3C07B34140C7F12006B84031
S31508008E50F1414140B1FBF3F603FB1611A2FB0645AF
S31508008E60001BA94102D2761E8018594180EA0102E8
S31508008E7021FA0EF3C7F1200462FA0EF20CFA07F093
S31508008E805A402CFA04F13043F0BD80EA010221FA77
S31508008E900EF3002162FA0EF260465A40F0BD8C4687
S31508008EA0B1FBF2F102FB11C31B0243EA1063B3FBE9
S31508008EB0F2FC02FB1C331B024CEA002043EA106357
S31508008EC0B3FBF2FC02FB1C331B024CEA002043EA0C
S31508008ED01063B3FBF2FC02FB1C331B024CEA0020B6
S31508008EE043EA1063B3FBF2FC02FB1C324CEA002097
S31508008EF00023704710F007003F4B1A684FF6FF0132
S31508008F000A403E4951EA00210A431A6070473A4826
S31508008F100068C0F302207047020052B2002A08D542
S31508008F200901374A40B210F00F00104400F8041C3B
S31508008F3003E00901334A40B21154704710B410F0E7
S31508008F400700D0F10703052B01D3042301E0D0F174
S31508008F500703041D072C01D2002000E0C01E0124CF
S31508008F6014FA03F35B1E1940814014FA00F0401E00
S31508008F701040084310BC704780B5411EB1F1807F90
S31508008F8001D301200EE0401E1F4908600F215FF043
S31508008F90FF30FFF7C1FF00201C49086007201C4965
S31508008FA00860002002BD80B5FFF7A4FF01BD70B5BB
S31508008FB004000D0016000020FFF7A9FF3200290063
S31508008FC0FFF7BCFF0100200040B2FFF7A5FF70BD08
S31508008FD080B5FFF7D1FF02BD042805D10C4801680A
S31508008FE051F00401016004E00948016831F0040108
S31508008FF001607047000000000CED00E00000FA0573
S3150800900018ED00E000E400E014E000E018E000E0FD
S3150800901010E000E080B500F001F801BD704730B4FB
S315080090200EE00268436802440830DC0744BFA9F131
S315080090300104E31852F8045B43F8045B091FF9D1ED
S3150800904050F8041B0029ECD130BC7047704700006B
S3150800905010B50400002C01D1012033E0A0690028D6
S31508009060FFD194F83900002805D1002084F838008B
S31508009070200000F05DFA242084F839002068C068D2
S3150800908030F400502168C860200000F0C7F8206856
S31508009090006930F49040216808612068406930F022
S315080090A02A00216848612068C06850F40050216889
S315080090B0C8600020E063202084F83900202084F866
S315080090C03A00002010BD2DE9FC4105000C00904631
S315080090D01F00002095F83A00202865D1002C03D0FF
S315080090E0404680B2002801D101205EE095F838009C
S315080090F0012801D1022058E0012085F83800002017
S31508009100E863222085F83A00FFF71CFB0600A5F85D
S315080091102C80A5F82E8005E028684068C005C00D9B
S315080091200880A41CE88D002836D0E88D401EE88506
S31508009130A868B0F5805F15D100973300002220217A
S31508009140280000F034F8002801D003202DE0210083
S3150800915028690028E0D02868406800F0FF000880E9
S31508009160641CDFE70097330000222021280000F066
S315080091701EF8002801D0032017E02869002804D12A
S31508009180286840682070641CCCE72868406810F09E
S315080091907F002070641CC5E7202085F83A0000206F
S315080091A085F83800002000E00220BDE8F6812DE9A8
S315080091B0F04105000E0090461F00069C28680068CE
S315080091C03040B04201D1012000E000204146C9B23A
S315080091D0884220D114F1010FF0D0002C04D0FFF7FB
S315080091E0B1FAC01B8442E9D22868C06830F4D0704E
S315080091F02968C860286840694008400029684861AD
S31508009200202085F83900202085F83A00002085F8C6
S315080092103800032000E00020BDE8F0812DE9F04188
S31508009220040000202068016931F44051E0680143D8
S31508009230206801612068C168BA480140A2682069AF
S31508009240024360690243E069024311432068C16032
S315080092502068416931F44071A06901432068416181
S31508009260E069B0F5004F40F0AE802068AE4988420C
S3150800927003D02068AD49884252D1FFF7DAFC804610
S31508009280FFF7D7FC0500FFF7D4FC0600FFF7D1FC73
S315080092900700FFF7CEFC6421192202FB08F8636871
S315080092A05B00B8FBF3F35FF0640CB3FBFCF35543C8
S315080092B0D4F804C05FEA4C0CB5FBFCF55643D4F869
S315080092C004C05FEA4C0CB6FBFCF65FF0640CB6FB18
S315080092D0FCF601FB1655ED0032356426B5FBF6F5AE
S315080092E06D0015F4F87515EB0315574363685B00B5
S315080092F0B7FBF3F302FB00F260684000B2FBF0F044
S315080093006422B0FBF2F001FB1031C8003230642150
S31508009310B0FBF1F010F00700451920688560FDE004
S31508009320FFF777FC8046FFF774FC0500FFF771FC32
S315080093300600FFF76EFC0700FFF76BFC6421192295
S3150800934002FB08F863685B00B8FBF3F35FF0640C94
S31508009350B3FBFCF35543D4F804C05FEA4C0CB5FBE9
S31508009360FCF55643D4F804C05FEA4C0CB6FBFCF691
S315080093705FF0640CB6FBFCF601FB1655ED003235C2
S315080093806426B5FBF6F56D0015F4F87515EB0315AF
S31508009390574363685B00B7FBF3F302FB00F26068B0
S315080093A04000B2FBF0F06422B0FBF2F001FB103192
S315080093B0C80032306421B0FBF1F010F007004519FF
S315080093C020688560AAE020685749884203D020684B
S315080093D05649884251D1FFF72CFC8046FFF729FCF5
S315080093E00500FFF726FC0600FFF723FC0700FFF73A
S315080093F020FC6421192202FB08F863689B00B8FB6D
S31508009400F3F35FF0640CB3FBFCF35543D4F804C0E4
S315080094105FEA8C0CB5FBFCF55643D4F804C05FEA4A
S315080094208C0CB6FBFCF65FF0640CB6FBFCF601FB95
S3150800943016552D0132356426B5FBF6F515F0F005FF
S3150800944015EB0315574363689B00B7FBF3F302FB61
S3150800945000F260688000B2FBF0F06422B0FBF2F024
S3150800946001FB1031080132306421B0FBF1F010F035
S315080094700F0045192068856050E0FFF7CAFB804653
S31508009480FFF7C7FB0500FFF7C4FB0600FFF7C1FBA4
S315080094900700FFF7BEFB6421192202FB08F8636880
S315080094A09B00B8FBF3F35FF0640CB3FBFCF3554386
S315080094B0D4F804C05FEA8C0CB5FBFCF55643D4F827
S315080094C004C05FEA8C0CB6FBFCF65FF0640CB6FBD6
S315080094D0FCF601FB16552D0132356426B5FBF6F56B
S315080094E015F0F00515EB0315574363689B00B7FBAA
S315080094F0F3F302FB00F260688000B2FBF0F064222E
S31508009500B0FBF2F001FB1031080132306421B0FBE8
S31508009510F1F010F00F00451920688560BDE8F0816C
S3150800952000000000F369FFFF00100140001401402D
S3150800953070470000BFF34F8FB6490A6812F4E0621D
S31508009540B54802430A60BFF34F8F00BFFDE780B5F9
S3150800955000F00DF800F0C2F801BD80B500F01BF868
S3150800956000F026F901BD80B5FFF7E4FF01BD80B51F
S31508009570AA48AB4901604FF461414160002181600E
S315080095800021C16000210161002181610C21416136
S31508009590FFF75EFD01BD70B5A24C2078002815D1F5
S315080095A0A14D280000F037F8012833D12878002883
S315080095B030D0287841282DDA00F05BF99B490860FD
S315080095C00120207000209A49087023E0984D964E95
S315080095D028783044401C00F01EF8012811D128785C
S315080095E0401C287028783178884213D100202070D2
S315080095F07078FF280ED1287802280BD1FFF7B3FF21
S3150800960008E000F036F9894909686431814201D2D7
S315080096100020207070BD80B50100002301227F481C
S31508009620FFF751FDC0B2002801D1012000E000205B
S3150800963002BDF8B504000D0016001F00FFF7E9FA91
S315080096404FF47A71B0FBF1F2002300E05B1C1800BE
S31508009650C0B2122840D2DFF8DCC1200080B219005F
S31508009660C9B21CF811E01900C9B20CEB41014978DE
S3150800967011EB0E0E1EF1010E0EFB00F0B2FBF0F11F
S3150800968000FB11200028E1D1210089B21800C0B2E0
S315080096901CF810E01800C0B20CEB4000407810EB44
S315080096A00E0E1EF1010E0EFB01F1B2FBF1F0288041
S315080096B028880028CAD0288840F201418842C5DA9D
S315080096C01800C0B21CF810003070DBB20CEB430077
S315080096D040783870012000E00020F2BD78B58BB0E4
S315080096E00020ADF8020000208DF8010000208DF85A
S315080096F0000040F267656B460DF101020DF10201AB
S315080097004FF4FA70FFF795FF4B4C4C4E266000203D
S3150800971020634B4860630020A0610020E0610020C0
S315080097202062002060620020A0620020E062002023
S31508009730A0600020E0609DF80100401E0004206142
S315080097409DF80000401E00056061BDF802006060DB
S315080097502000FEF719FD002D02D46D05394805E0F5
S3150800976025F00045ED0055F0040537482168B1425B
S3150800977002D10021069101E00E21069100210791F0
S31508009780012108912900090C0191ADB20295010049
S31508009790090C039180B204900020059001200990DD
S315080097A00E200A9001A92000FEF7C1FD0CB070BD7D
S315080097B070B540F2676600251F4C00220021200084
S315080097C0FEF736FE002823D1002E09D4606B006808
S315080097D0B04210D1606B806800280CD101250AE0E0
S315080097E026F00046606B4068B04204D1606B806822
S315080097F0042800D10125EDB2012D09D1606B007D49
S31508009800FF2805D1606B0069022801D1FFF7ABFE7E
S3150800981070BD00000CED00E00400FA058C00002085
S3150800982000480040FD00002004000020F000002051
S31508009830FC000020D09D000848000020006400407D
S31508009840CC0000200400E0FFFCFF1F0080B5FFF7F6
S31508009850DDF94FF47A71B0FBF1F0FFF7B9FB04209C
S31508009860FFF7BAFB002200215FF0FF30FFF79FFBEE
S3150800987001BD80B5FEF766FF02BD80B500F004F8AD
S31508009880FFF7C8FB01BD000002480168491C0160DA
S31508009890704700BFF8000020F8B40022002200221A
S315080098A0002337E0092704E0DFF8E8219042F9D1E0
S315080098B00827FFB213F00302D2B2920097403E4344
S315080098C01A00920845F82260DFF8CC512A68A243AC
S315080098D04E68F60300D522432A60DFF8C0512A688D
S315080098E0A2434E68B60300D522432A60DFF8B0517A
S315080098F02A68A2434E68F60200D522432A60DFF89A
S31508009900A4512A68A2434E68B60201D51443220020
S315080099102A605B1C102B80F0B080012515FA03F233
S315080099200C6814409442F4D14A68022A02D04A6864
S31508009930122A17D11A00D20800EB8202166A0F27DC
S3150800994013F00702D2B292009740BE430F6913F094
S315080099500702D2B2920097403E431A00D20800EBA3
S3150800996082021662076803261A00D2B2520016FA55
S3150800997002F2974391F804C01CF0030C1A00D2B205
S3150800998052001CFA02FC5CEA070707604A68012ACB
S3150800999008D04A68022A05D04A68112A02D04A68BD
S315080099A0122A19D187681A00D2B2520016FA02F2A0
S315080099B09743D1F80CC01A00D2B252001CFA02FC26
S315080099C05CEA0707876042689D40AA434D68C5F36D
S315080099D000159D402A434260C5681A00D2B252005B
S315080099E09640B5438E681A00D2B252009640354367
S315080099F0C5604A68D2008CD5002200922A4A1568AA
S31508009A0055F480451560126812F480420092009A57
S31508009A10264D1A00920855F822600F2713F0030204
S31508009A20D2B292009740BE43214A904201D1002704
S31508009A303FE7204A904201D101273AE71E4A904261
S31508009A4001D1022735E71D4A904201D1032730E7A5
S31508009A501B4A904201D104272BE71A4A904201D1AA
S31508009A60052726E7184A904201D1062721E7174A13
S31508009A7090427FF419AF07271BE7F1BC7047D2B2B3
S31508009A80002A02D089B2816102E089B209048161A3
S31508009A907047000000200240003C0140043C0140A1
S31508009AA0083C01400C3C014044380240083801405B
S31508009AB0000002400004024000080240000C024078
S31508009AC0001002400014024000180240001C024028
S31508009AD080B500F007F8FFF73AFD00F0F9F8FFF750
S31508009AE03CFDFAE780B500F009F800F019F900F036
S31508009AF009F8FFF7ABFE00F0E3F801BD68486949CD
S31508009B000860704700B591B00120059001200690C5
S31508009B1002200B905FF480000C9019200D90F02025
S31508009B200E9002200F900520109005A8FEF710FE53
S31508009B30002800D0FEE70F200090022001900020A8
S31508009B4002904FF4A05003904FF4805004900321E4
S31508009B506846FEF77EFF002800D0FEE711B000BD7C
S31508009B6010B586B0002005904F48016851F4804131
S31508009B700160006810F48040059005980020059063
S31508009B804A48016851F002010160016811F00201BA
S31508009B900591059900210591016851F008010160B8
S31508009BA0016811F0080105910599002105910168E0
S31508009BB051F020010160006810F02000059005981A
S31508009BC0002005903A48016851F480210160016837
S31508009BD011F480210591059900210591016851F03C
S31508009BE000710160006810F0007005900598032068
S31508009BF0FFF7D9F9002200217FF00B00FFF7D7F90C
S31508009C00002200217FF00A00FFF7D1F90022002187
S31508009C107FF00900FFF7CBF9002200217FF004004E
S31508009C20FFF7C5F9002200217FF00300FFF7BFF90F
S31508009C30002200217FF00100FFF7B9F90022002178
S31508009C405FF0FF30FFF7B3F94FF480700090012002
S31508009C500190012002900120039069461548FFF7FC
S31508009C601BFE4FF4407400940220019001200290DC
S31508009C70032003900720049069460F48FFF70CFE5F
S31508009C8000940220019000200290032003900920EE
S31508009C90049069460948FFF7FFFD06B010BD0000AD
S31508009CA00080000808ED00E04438024030380240E1
S31508009CB04038024000140240000C024000040240F2
S31508009CC080B500224FF480711248FFF7D8FE01BD17
S31508009CD038B5FFF7CEFD04000F4D2868201AB0F5F9
S31508009CE0FA7F15D30D490878002808D10120087095
S31508009CF001224FF480710748FFF7C1FE07E00020F4
S31508009D00087000224FF480710248FFF7B8FE2C60F5
S31508009D1031BD000000140240F4000020FE000020BF
S31508009D2080B50B48016851F400710160016851F46F
S31508009D3080610160016851F4807101600320FFF7BA
S31508009D4032F90020FEF7AAFFFFF70AFF002002BD3E
S31508009D50003C02400D49086850F0010008600020E8
S31508009D600B4A10600A680B4802400A600A480B4A08
S31508009D701060086830F480200860002008490860F0
S31508009D805FF000600749086070470000003802402D
S31508009D9008380240FFFFF6FE10300024043802405F
S31508009DA00C38024008ED00E010B50749794418312F
S31508009DB0064C7C44163404E00A68081D114488479A
S31508009DC00146A142F8D110BD2C0000004C0000004D
S31508009DD005020602060307030803090309040A0421
S31508009DE00B040C040C050D050E050F050F061006D1
S31508009DF01007100817E9FFFFFC0000000400002008
S31508009E00000000001BF2FFFF04000000F401000040
S31508009E10000000200000000000F00DF8002801D026
S31508009E20FFF7C2FFAFF300800020AFF30080FFF713
S31508009E304FFE00F002F80120704700F001B800005C
S31508009E400746384600F002F8FBE7000080B5AFF396
S31508009E500080024A11001820ABBEFBE7260002006C
S31508009E600248854602488047024800470009002004
S31508009E70559D0008899E00080000000000000000AB
S31508009E800102030406070809AFF30080AFF3008058
S31508009E90FFF7C2FF0000000001020304FFF7FEBF40
S31508009EA0FFF7FEBFFFF7FEBFFFF7FEBFFFF7FEBFD8
S31508009EB0FFF7FEBFFFF7FEBFFFF7FEBFFFF7FEBFC8
S31508009EC0FFF7FEBFFFF7FEBFFFF7FEBFFFF7FEBFB8
S31508009ED0FFF7FEBFFFF7FEBFFFF7FEBFFFF7FEBFA8
S31508009EE0FFF7FEBFFFF7FEBFFFF7FEBFFFF7FEBF98
S31508009EF0FFF7FEBFFFF7FEBFFFF7FEBFFFF7FEBF88
S31508009F00FFF7FEBFFFF7FEBFFFF7FEBFFFF7FEBF77
S31508009F10FFF7FEBFFFF7FEBFFFF7FEBFFFF7FEBF67
S31508009F20FFF7FEBFFFF7FEBFFFF7FEBFFFF7FEBF57
S31508009F30FFF7FEBFFFF7FEBFFFF7FEBFFFF7FEBF47
S31508009F40FFF7FEBFFFF7FEBFFFF7FEBFFFF7FEBF37
S31508009F50FFF7FEBFFFF7FEBFFFF7FEBFFFF7FEBF27
S31508009F60FFF7FEBFFFF7FEBFFFF7FEBFFFF7FEBF17
S31508009F70FFF7FEBFFFF7FEBFFFF7FEBFFFF7FEBF07
S31508009F80FFF7FEBFFFF7FEBFFFF7FEBFFFF7FEBFF7
S31508009F90FFF7FEBFFFF7FEBFFFF7FEBFFFF7FEBFE7
S31508009FA0FFF7FEBFFFF7FEBFFFF7FEBFFFF7FEBFD7
S31508009FB0FFF7FEBFFFF7FEBFFFF7FEBFFFF7FEBFC7
S31508009FC0FFF7FEBFFFF7FEBFFFF7FEBFFFF7FEBFB7
S31508009FD0FFF7FEBFFFF7FEBFFFF7FEBFFFF7FEBFA7
S31508009FE0FFF7FEBFFFF7FEBFFFF7FEBFFFF7FEBF97
S31508009FF0FFF7FEBFFFF7FEBFFFF7FEBFFFF7FEBF87
S3090800A0000024F40036
S70508009E89CB
